:020000040000FA
:040000000FEF00F00E
:0400080098EF06F077
:08001800100098EF06F0130E32
:10002000926E0F0EC16E020E936E900E946E020EC3
:10003000D56ED58CD59AD596806A816A826AC76A50
:10004000C00EC76EC66A210EC66E006A016A026AD9
:10005000036A046A676A686A828C8294236A050E5E
:10006000246E93EC06F0809A808A040E0C6EFA0ED1
:100070000A6ED1EC06F00C2EFAD7809A81A21DEC04
:1000800004F0056A046AC3EC03F063B0028263B251
:10009000028463B4028863B6028A63B8028C63BACE
:1000A000058C02B282EC01F08284BDEC02F05AECC5
:1000B00002F0D58EF28AF28EF28E808AFA0E0A6EE5
:1000C000D1EC06F0C5EC05F0040003B08BEC00F0B9
:1000D00004B2A5D703B05AEC02F003B2B0EC00F0C2
:1000E000000000001AEC05F0DBEC04F087EC00F0F7
:1000F0000000000002BE05D06B66E6D7B4EC01F04C
:10010000E3D7029E68C067F0D2EC01F0DDD704AC03
:100110001200049C1200000E4D6E150E4E6EA6ECE1
:1001200002F0C9CF07F007BE0DD007BC15D0040EF2
:100130004D6E020E4E6EA6EC02F0C9CF07F007B668
:100140000DD0120004B007D00480000ED56ED58CFF
:10015000D59AD596D58E1200048212000482120020
:100160000392040E4D6E260E4E6EA6EC02F0C9CF21
:100170004FF04E2AA6EC02F0C9CF50F0506601D0E5
:10018000120093EC06F05050410E505CD8B083D171
:10019000600E4D6E000E4E6EEA6A00EE6CF050C0BE
:1001A00069F0A6EC02F0C9CFEFFF4E2AE92A692ECA
:1001B000F8D7FF0E6C5C02E04BEF02F0AA0E6D5C0C
:1001C00002E04BEF02F0C80E6F5C0DE0CA0E6F5CF0
:1001D00053E0CE0E6F5C6AE0030E6F5C02E173EFDA
:1001E00001F04BEF02F06E6AC90E6F6E73C075F0CE
:1001F00074C076F0FF0E736EFF0E746E010E776E94
:10020000010E786E000E300F7A6E000E300F7B6E8E
:10021000030E300F7C6E640E7D6E51C07EF052C0B6
:100220007FF053C080F054C081F055C082F056C0BA
:1002300083F057C084F058C085F059C086F05AC08A
:1002400087F05BC088F05CC089F05DC08AF05EC05A
:100250008BF05FC08CF060C08DF061C08EF062C02A
:100260008FF063C090F064C091F065C092F0270EEB
:100270006A6E6AC070F09BD0600E4D6E0E0E4E6EB0
:1002800000EE51F0EA6A190E0C6EA6EC02F0C9CF2E
:10029000EFFFE92A4E2A0C2EF8D76E6AF00E6F6E29
:1002A0000E0E6A6ED7EC01F082EC04F06E6ACE0E90
:1002B0006F6E9BEC01F0010E776E010E786E66C0DA
:1002C0007AF067C07BF005B42E8E2EC07CF02FC074
:1002D0007DF005B6308E30C07EF031C07FF00296E2
:1002E000140E6A6E64D07AC066F082EC01F09BEC6A
:1002F00001F066C07AF002B2A5EC01F00F0E6A6E52
:1003000056D0120066A804D066B0828066A08290A3
:1003100066AA04D066B2828266A2829266AC04D0DB
:1003200066B4808466A4809466AE120066B6808649
:1003300066A680961200666A82B0668082B2668285
:1003400080B4668480B66686120066B0668866B23F
:10035000668A66B4668C66B6668E0F0E456E66C09B
:1003600044F080EC06F0120002A401D002A6676AF5
:1003700080A0678080A26782938093840000000041
:1003800081A4678481A06786028602BA01D0120028
:100390006750685C01E1120067C068F002AC02D0EF
:1003A000020E6B6E03846E6A6A0E6F6E82D703A4B0
:1003B00010D075EC03F099EC03F0040E4B6E010EB7
:1003C0004C6E010E4A6EAEEC03F0040E4A6EAEECBB
:1003D00003F0040E4D6E240E4E6EA6EC02F0C9CF53
:1003E0001CF01CC048F04E2AA6EC02F0C9CF1BF04E
:1003F0001BC049F01E6A6AC01DF048C01CF049C00D
:100400001BF06FEC06F0040E4B6E240E4C6E1CC0FD
:100410004AF0AEEC03F04C2A1BC04AF0AEEC03F0FD
:10042000070E4816FF0E491648C01CF049C01BF0C5
:10043000400E1E6E1D6A6FEC06F01CC048F01BC01B
:1004400049F048C04BF049C04CF06AC00CF000EED7
:100450006CF0EA6AEFCF4AF0AEEC03F04FEC02F03A
:10046000E92A0C2EF7D7F29E040E4B6E010E4C6E4D
:10047000200E4A6EAEEC03F05AEC02F003A40BD04F
:100480000394040E4B6E010E4C6E080E4A6EAEECD9
:1004900003F0BDEC02F099EC03F0F28E12004C2A4E
:1004A000D8B04B2A480E4B5C01E01200400E4B6E58
:1004B0004C6A12004DC046F04EC047F004940390C1
:1004C000040E4D6E030E4E6EA6EC02F0C9CF1BF06B
:1004D000000E1B5C04E10484000E086E2CD0010E9B
:1004E0001B5C03E1090E086E26D0130E1B5C03E1B2
:1004F000010E086E20D0140E1B5C0AE10290020E61
:10050000086E19D0150E1B5C03E10A0E086E13D09D
:10051000170E1B5C06E1A0EC02F0030E086E0382CE
:100520000AD01C0E1B5C05E1040E086E99EC03F06A
:1005300002D0050E086E46C04DF047C04EF01200C6
:1005400002B012000A0E106E02801200829C00009F
:1005500000000F0EC96E46EC06F04DC0C9FF46EC18
:1005600006F04EC0C9FF46EC06F0AA0EC96E46EC76
:1005700006F0C7A0FED7828C120046EC06F046ECCF
:1005800006F04B6A4C6A800E4A6EAEEC03F04C2AC1
:1005900055C04AF0AEEC03F04C2A56C04AF0AEEC1F
:1005A00003F04C2A57C04AF0AEEC03F04C2A58C076
:1005B0004AF0AEEC03F04C2A59C04AF0AEEC03F01E
:1005C0004C2A5AC04AF0AEEC03F04C2A5BC04AF009
:1005D000AEEC03F04C2A5CC04AF0AEEC03F04C2ABF
:1005E00054C04AF0AEEC03F04C2A200E4A6EAEEC3A
:1005F00003F04C2A180E4A6EAEEC03F04C2A1B0E88
:100600004A6EAEEC03F04C2A150E4A6EAEEC03F0C7
:100610004C2A5F0E4A6EAEEC03F04C2A51C04AF0F1
:10062000AEEC03F04C2A52C04AF0AEEC03F04C2A78
:1006300053C04AF0AEEC03F04C2A54C04AF0AEEC82
:1006400003F0040E4B6E4C6A010E4A6EAEEC03F0E2
:10065000040E4B6E040E4C6E61C04AF0AEEC03F01B
:100660004C2A62C04AF0AEEC03F0000E4B6E1A0E3C
:100670004C6E550E4A6EAEEC03F0000E4B6E1B0E28
:100680004C6E550E4A6EAEEC03F0000E4B6E160E1D
:100690004C6E010E4A6EAEEC03F0040E4B6E0C0E67
:1006A0004C6E5DC04AF0AEEC03F04C2A5EC04AF0DE
:1006B000AEEC03F04C2A5FC04AF0AEEC03F04C2ADB
:1006C00060C04AF0AEEC03F04C2A61C04AF0010E63
:1006D0004A6EAEEC03F04C2A540E4A6EAEEC03F0B8
:1006E00099EC03F046EC06F01200040E4B6E100E6F
:1006F0004C6E010E010E4A6EAEEC03F04C2A540E05
:10070000550E4A6EAEEC03F046EC06F0120004946F
:10071000040E4B6E010E4C6E100E4A6EAEEC03F0E2
:10072000010E4A6EAEEC03F0020E4A6EAEEC03F020
:1007300012000494040E4B6E010E4C6E100E4A6EA5
:10074000AEEC03F003A401D01200010E4A6EAEEC31
:1007500003F0020E4A6EAEEC03F01200829C000021
:100760000000F00EC96E46EC06F04BC0C9FF46EC27
:1007700006F04CC0C9FF46EC06F04AC0C9FF46EC83
:1007800006F0828C1200456A77EC06F044C051F006
:1007900077EC06F044C052F077EC06F044C053F01A
:1007A00077EC06F044C054F077EC06F044C055F006
:1007B00077EC06F044C056F077EC06F044C057F0F2
:1007C00077EC06F044C058F077EC06F044C059F0DE
:1007D00077EC06F044C05AF077EC06F044C05BF0CA
:1007E00077EC06F044C05CF077EC06F044C05DF0B6
:1007F00077EC06F044C05EF077EC06F044C05FF0A2
:1008000077EC06F044C060F077EC06F044C061F08D
:1008100077EC06F044C062F077EC06F044C063F079
:1008200077EC06F044C066F077EC06F044C064F064
:1008300077EC06F044C065F01200456AC00E446EC5
:1008400080EC06F0A80E446E80EC06F01C0E446EA0
:1008500080EC06F0010E446E80EC06F0C00E446E93
:1008600080EC06F0A80E446E80EC06F01C0E446E80
:1008700080EC06F0FE0E446E80EC06F0FF0E446E37
:1008800080EC06F0FF0E446E80EC06F0FF0E446E26
:1008900080EC06F0000E446E80EC06F0C00E446E54
:1008A00080EC06F0A80E446E80EC06F01C0E446E40
:1008B00080EC06F00B0E446E80EC06F0010E446EE8
:1008C00080EC06F0540E446E80EC06F0080E446E88
:1008D00080EC06F0000E446E80EC06F0040E446ED0
:1008E00080EC06F0020E446E80EC06F0140E0C6EE6
:1008F000320E0A6ED1EC06F0807A0C2EF9D781A266
:10090000F5D71200456A51C044F080EC06F052C0A1
:1009100044F080EC06F053C044F080EC06F054C084
:1009200044F080EC06F055C044F080EC06F056C070
:1009300044F080EC06F057C044F080EC06F058C05C
:1009400044F080EC06F059C044F080EC06F05AC048
:1009500044F080EC06F05BC044F080EC06F05CC034
:1009600044F080EC06F05DC044F080EC06F05EC020
:1009700044F080EC06F05FC044F080EC06F060C00C
:1009800044F080EC06F061C044F080EC06F062C0F8
:1009900044F080EC06F063C044F080EC06F0452A99
:1009A00064C044F080EC06F065C044F080EC06F0D2
:1009B0000FEF00F0120005AC3CD030C01CF031C08D
:1009C0001BF02EC01EF02FC01DF05EEC06F0D8B05C
:1009D0002FD02EC01CF02FC01BF01E6A64C01DF06B
:1009E0006FEC06F01CC01EF01BC01DF030C01CF0E8
:1009F00031C01BF05EEC06F0D8B002D0808419D074
:100A00002EC01CF02FC01BF01E6A65C01DF06FECDD
:100A100006F01CC01EF01BC01DF030C01CF031C021
:100A20001BF05EEC06F0D8B003D080A401D001D05A
:100A300080941200010E235C04E00A0E235C26E081
:100A400012000590059205940596C6EC05F0100E6F
:100A5000325C06E0280E325C03E00580236A120057
:100A6000100E3B5C04E0280E3B5C01E00582DFECED
:100A700005F0CC0E256E12EC06F0080E3DEC06F0EB
:100A8000440E256E12EC06F0232A1200236ADFECD6
:100A900005F0CC0E256E12EC06F0BE0E256E12ECA3
:100AA00006F0EDEC05F026C02BF027C02DF0EDECA4
:100AB00005F026C02AF027C02CF032C029F02AC049
:100AC0001CF02BC01BF086EC05F001BA058405A0D4
:100AD00003D01C6A1B6A05941CC02EF01BC02FF0AB
:100AE0002CC01CF02DC01BF03BC029F086EC05F09B
:100AF00001BA058605A203D01C6A1B6A05961CC0B4
:100B000030F01BC031F0236A01881200019A1CAE3C
:100B10000ED0018A1C1E1B1E1CC01EF01BC01DF027
:100B2000010E6FEC06F01EC01CF01DC01BF0100E75
:100B3000295C04E0280E295C11E012001C6A019275
:100B40001BB00182D8901B324EEC06F001A21200BD
:100B5000050E1D6E1E6A6FEC06F012002BC044F0ED
:100B60000F0E4416040E0C6ED8901C321B320C2E45
:100B7000FBD71C6A4EEC06F0445080EC19F01D6E59
:100B80001E6A6FEC06F012001200236ADFEC05F01B
:100B9000330E256E12EC06F0080E286E10EE32F0C1
:100BA000E26A20EE3BF0DA6AEDEC05F026C0E7FFE2
:100BB000E12A27C0DFFFD92A282EF6D71200460ED9
:100BC0003DEC06F031EC06F0460E3DEC06F036EC5E
:100BD00006F0500E3DEC06F01200080E0C6E266A70
:100BE000276A31EC06F00000000036EC06F0000049
:100BF0000000000000000000000000008250076EAE
:100C000007AED89007BED88026328050076E07A85E
:100C1000D89007B8D8802732040E3DEC06F00C2E91
:100C2000E0D71200080E0C6E2532D8A004D00ED0EA
:100C30000C2EFAD7120031EC06F0080E3DEC06F04F
:100C400036EC06F0010E3DEC06F0F2D731EC06F082
:100C5000010E3DEC06F036EC06F0090E3DEC06F018
:100C6000E7D7829E949E809892981200828E948EEE
:100C7000828E80889288808812000A6E090E0B6E20
:100C800004000B2EFDD70A2EF9D7000C190E0A6EA0
:100C90000000000000000A2EFBD712001CC01EF04E
:100CA0001BC01DF0030E0C6ED8901B361C360C2E8C
:100CB000FBD76FEC06F06FEC06F012001F6A1D50B8
:100CC0001B5ED8B004D0010E1C5ED8A01F801E5041
:100CD0001C5ED8A01F80D8901FB0D88012001D5075
:100CE0001B261E50D8B01E3C1C2612001200455078
:100CF000A96EA69EA69CA680A850446E452A120006
:100D0000A1984550A96E4450A86EA69EA684F29E56
:100D1000550EA76EAA0EA76EA682A1A88DEF06F0AB
:100D2000452AF28E1200010E216EBA0E226E1200BA
:100D3000F2B49DEF06F0CFEF06F00F2E30D00E6626
:100D40000BD0030E0E6EE80E0F6E807A6B6601D02C
:100D500007D06B4E028E04D00E06FF0E0F6E0CD025
:100D600002A80AD0226607D0216602D0048204D0ED
:100D70002106FF0E226E2206048C038002A004D0FE
:100D8000102E02D0048202900B0E235C02E3090EA7
:100D9000236E232A04D0242E02D0050E246EF29452
:100DA00011000A6E0A6601D017D0960E04000000EA
:100DB0000000000000000000000000000000000033
:100DC00000000000000000000000FF0FD8A4D6EFD4
:100DD00006F00A2ED5EF06F012000A6E00000000A1
:0C0DE0000000000000000A2EF9D71200ED
:10330000076E330EFA6E0752F924D8B0FA2A060F68
:10331000D8B0FA2A07460750F926000C010C010C18
:10332000020C020C030C030C040C050C050C060C1F
:0A333000060C070C080C080C090C31
:020000040030CA
:03000100021E1FBD
:020005008181F7
:060008000FC00FE00F40E5
:0200000400F00A
:10000000C0A81C01C0A81CFEFFFFFF00C0A81C0B5D
:0600100001540000281459
:00000001FF
